:100000000C9446000C945D000C945D000C945D0013
:100010000C945D000C945D000C945D000C945D00EC
:100020000C945D000C945D000C945D000C945D00DC
:100030000C945D000C945D000C945D000C945D00CC
:100040000C945D000C945D000C945D000C945D00BC
:100050000C945D000C945D000C945D000C945D00AC
:100060000C945D000C945D000C945D000C945D009C
:100070000C945D000C945D000C945D000C945D008C
:100080000C945D000C945D000C945D0011241FBE67
:10009000CFEFD0E4DEBFCDBF11E0A0E0B1E0E2EAF7
:1000A000F5E000E00BBF02C007900D92A031B10750
:1000B000D9F70E94CA020C94CF020C940000089A4F
:1000C00092B181E0892782B92FEF8FEF9CE2215016
:1000D00080409040E1F700C000000895A0E8B0E043
:1000E0008C9183608C93E1E8F0E08081886180836B
:1000F0008C9180628C9380818360808380E490E027
:10010000909389008093880089E390E090938B001E
:1001100080938A00549A08950E946E000E943301D1
:100120000E94A9012FEF8FEF9CE221508040904068
:10013000E1F700C000000E94A90180E091E00C946A
:100140003D0217B817B82898299A2A9A000080E526
:1001500093EC1F9B02C00197E1F742988FEF87B99C
:100160000895CF93DF9300D0CDB7DEB7442331F0AD
:100170006A8389830E94A10089816A8165B981307F
:1001800011F4289A01C02898299800002A9A0000A2
:100190002A980F900F90DF91CF91089541E00C9431
:1001A000B100482F50E0DA01B595A795EA2FE1702C
:1001B000F0E0EE0FFF1FDA01B595A795B595A7956D
:1001C0002A2F217030E0220F331F220F331F2E2BD6
:1001D0008170822B73E0559547957A95E1F7642FEE
:1001E000617070E0E3E0660F771FEA95E1F7862B18
:1001F00008958F700E94D10098B1907F892B88B9A3
:100200000895CF93C82F442321F081E28A95F1F716
:100210000000862F807F0E94F900C13011F4289AD7
:1002200001C02898299800002A9A00002A98CF91A6
:10023000089586B196B146B136B19270292F220F3A
:10024000942F9470990F990F922B8170982B832F74
:100250008870880F880F880F892B0895389A399AEB
:100260003A9A3B9A089584B1876084B90C942E0120
:10027000389839983A983B980895882311F0289A2D
:1002800001C02898299A0E9438012A9A000095B145
:100290002A9800002A9A000025B12A982F70892FE9
:1002A0008295807F822B0895CF93DF9380E00E9418
:1002B0003D01C9EED3E087FF06C0219721F080E021
:1002C0000E943D01F8CFDF91CF910895CF93DF9346
:1002D000D82FC62F41110E9454010E942E018C2F4D
:1002E00082958F700E94F900D13011F4289A01C0D4
:1002F0002898299800002A9A00002A988C2F8F703D
:100300000E94F90000002A9A00002A98DF91CF91FC
:10031000089541E00C946601611102C060E801C0DB
:1003200060EC8F73682B80E00C94890161E080E0C1
:100330000E9489018BE791E00197F1F700C000006E
:10034000089568E180E00C94890162E080E00C94FB
:100350008901CF93DF932A982898299880E00E94FA
:10036000F9002FE38DE093E0215080409040E1F7C9
:1003700000C00000C3E0D0E040E060E080E00E9408
:1003800001018FE493EC0197F1F700C00000219781
:1003900099F740E060E280E00E9401019FE32DE0D8
:1003A00083E0915020408040E1F700C0000040E031
:1003B00068E280E00E94660140E068E280E00E941E
:1003C000660140E068E280E00E94660140E068E289
:1003D00080E00E94660140E068E280E00E946601E1
:1003E00040E068E280E00E9466019FE021E281E057
:1003F000915020408040E1F700C0000040E067E1FC
:1004000080E00E9466019FE021E281E0915020405F
:100410008040E1F700C0000040E06CE080E00E9416
:1004200066019FE021E281E0915020408040E1F7A9
:1004300000C0000040E061E080E00E94660187E8C3
:1004400093E10197F1F700C0000040E066E080E032
:100450000E94660187E893E10197F1F700C0000070
:10046000DF91CF91089540E068E080E00C94660150
:1004700040E06CE080E00C946601CF92DF92EF9256
:10048000FF920F931F93CF93DF938C010E94A501DE
:100490002FE986E891E0215080409040E1F700C0CC
:1004A00000000E949601EFE9F6E821E0E150F040FB
:1004B0002040E1F700C0000060E880E00E94890170
:1004C00089EF90E00197F1F700C00000F80101907A
:1004D0000020E9F73197E01BF10BE930F10508F056
:1004E000E8E07801CE2FD0E0C701801B910B8C177C
:1004F0009D0774F4E1EEF4E03197F1F700C00000DD
:10050000F70161917F0140E081E00E946601ECCF3C
:10051000F80101900020E9F73197E01BF10B3997C2
:1005200080F1FFE926E881E0F15020408040E1F7CA
:1005300000C0000060EC80E00E948901680198E042
:10054000C90ED11CE12CF12CF80101900020E9F733
:100550003197E01BF10BEC1BFD0BEE16FF0688F448
:10056000E1EEF4E03197F1F700C00000F60161918F
:100570006F0140E081E00E946601FFEFEF1AFF0A81
:10058000E3CFDF91CF911F910F91FF90EF90DF901C
:10059000CF9008950E948C000E945F00FDCFF894D8
:0205A000FFCF8B
:1005A200747774723A2040736F6C696E6975730068
:00000001FF
